:100000000C94DB000C9413010C9413010C94130159
:100010000C9413010C9413010C9413010C94130110
:100020000C9413010C9413010C9413010C94800A8A
:100030000C943C0A0C947F0B0C9413010C94130148
:100040000C9413010C9413010C9413010C944D0B9C
:100050000C9413010C9413010C9413010C941301D0
:100060000C9413010C9413010C9413010C941301C0
:100070000C941301640464049F049F04D004C80515
:10008000C805C805EC0460057105710559088008AC
:10009000140A8008140AC808EB08140AD609E909EA
:1000A00005010980A101850319012AB70015012660
:1000B000B700950175108100C0050C0901A10185EB
:1000C0000419012AA002150126A0029501751081CC
:1000D00000C005010906A101050719E029E715007F
:1000E00025019508750181029501750881010507B3
:1000F000190029FF150026FF0095067508810005E7
:10010000081901290595057501910295017503915D
:1001100001C009023B00020100A0FA09040000012D
:10012000030101000921110100012240000705819E
:100130000308000109040100010300000009211166
:100140000100012232000705820320000112010094
:1001500002000000080DF000000100010200012271
:10016000036600720061006E006B00690065005F4D
:10017000006D006100630072006F00700061006438
:10018000000000140345007200690063002000575E
:10019000006F006F00640000000403090400000009
:1001A000004A00A800BE00BD0000000000AC00AE88
:1001B00000AB0000000011241FBECFEFD2E0DEBF75
:1001C000CDBF04B603FE18C08091E9019091EA0109
:1001D000A091EB01B091EC018730904BA740B04B60
:1001E00059F41092E9011092EA011092EB01109279
:1001F000EC01E0E0F8E1099511E0A0E0B1E0E2E413
:10020000F9E202C005900D92AA35B107D9F721E0B5
:10021000AAE5B1E001C01D92A93EB207E1F70E9434
:100220004F110C949F140C940000990F990F890F93
:10023000A82FA77086958695869590E063E070E07C
:100240000E945314FC01E45AFE4F40E050E080E06D
:10025000219130E00A2E02C0369527950A94E2F7E4
:1002600021703327042E01C0220F0A94EAF7822B53
:100270004F5F5F4F4330510559F70895262F990F6F
:10028000990F890F982F9770A1E001C0AA0F9A9536
:10029000EAF786958695869590E063E070E00E9487
:1002A0005314FC01E45AFE4F40E050E0622F70E02E
:1002B00090819B01042E02C0369527950A94E2F79F
:1002C0002170219529272A23292721934F5F5F4FEA
:1002D0004330510569F70895882341F08095909146
:1002E00070018923809370010C94E80E089588238F
:1002F00039F090917001892B809370010C94E80E75
:10030000089580E090E00E94BE0B80E090E00E94A3
:10031000A80B1092CF010C94E80E8093D8010C9496
:10032000810121E030E001C0220F8A95EAF7209593
:100330008091D80182230C948D0121E030E001C02E
:10034000220F8A95EAF78091D801822B0C948D01B7
:100350008823A9F19CEF980F913A60F4E7E8F1E067
:100360009281891301C01282319641E0ED38F40781
:10037000B9F714C090E2980F983090F4877021E09C
:1003800030E0A90102C0440F551F8A95E2F7CA0167
:100390008095909170018923809370010C94E80EF0
:1003A0009BE5980F933020F480E090E00C94BE0B16
:1003B000885A873120F480E090E00C94A80B0895CF
:1003C0000F931F93CF93882309F46EC09CEF980F6F
:1003D000913A58F5C82F09E811E08FE891E0F8014B
:1003E0002191C21721F08E179F07D1F70EC0E7E8C1
:1003F000F1E08DE891E02281C21301C012823196B2
:100400008E179F07C1F70E94E80EEFEF80E0D8013A
:100410009D918D01C917E1F0EF3F19F4911101C0D1
:10042000E82F8F5F863099F736C090E2980F9830AA
:10043000A0F4877021E030E0A90102C0440F551FED
:100440008A95E2F7CA0190917001892B809370011F
:10045000CF911F910F910C94E80EEBE5E80FE3307C
:1004600050F4F0E0E35FFE4F808190E0CF911F9168
:100470000F910C94BE0B885A8731B0F4E82FF0E04E
:10048000EE0FFF1FE05FFE4F80819181CF911F91A2
:100490000F910C94A80BEF3FD9F20E2E000CFF0B1E
:1004A000E957FE4FC283D4CFCF911F910F9108958A
:1004B000CF92DF92EF92FF920F931F93CF93DF9330
:1004C0000091D8012091D001022BC7E0D0E010E0CC
:1004D000C92ED12CE82EF12CC8010C2E02C0959506
:1004E00087950A94E2F780FD04C02197A8F780E081
:1004F00019C0CE0163E070E00E9453148C0D9D1D65
:10050000FC01EE0FFF1FEE0FFF1FEE0DFF1DEE0FA4
:10051000FF1FE356FE4F859194910E94030D0197B2
:1005200021F38C2FDF91CF911F910F91FF90EF90CE
:10053000DF90CF9008958093D0010C948101FC014D
:10054000808191810E94820F92959F70963079F000
:1005500010F4925001C09A50923068F4803F69F0D4
:1005600018F4883E40F409C0843F29F406C0883E50
:1005700020F0813F11F080E0089581E0089586E049
:10058000E9E8F1E0DF011D928A95E9F70C94810119
:100590001F93CF93DF93182FEB010E94E001209768
:1005A00041F08FE99FE00197F1F700C0000021972B
:1005B000F6CF812FDF91CF911F910C94A801CF939B
:1005C000DF93CDB7DEB767970FB6F894DEBF0FBEE7
:1005D000CDBF4B8B5C8B6D8B7E8B8F8B61111092A3
:1005E000CF0186E09E01235F3F4FD901E82F1D9286
:1005F000EA95E9F795E0FE017396D90101900D9215
:100600009A95E1F79C894E895F897B897D879E87D2
:100610006F87598B488BF901DE01179601900D9277
:100620008A95E1F7CE0107960E94A00F811153C071
:1006300086E0FE013796DE01119601900D928A95B3
:10064000E1F7FF81E8856A857B856115710531F0E9
:10065000EF3F31F481E0FF3F19F403C081E001C0B6
:1006600080E080FD38C08091950190E09C012F5F73
:100670003F4F277033274091C60150E024173507BC
:1006800089F1F983EA837D836C8366E070E00E94E0
:100690005314DC01AA56BE4F96E0FE01319601903C
:1006A0000D929A95E1F7209395010E940F0F13C0C8
:1006B00090E066E070E00E9453148A569E4F0E94BC
:1006C000A00F8823F1F08091C60190E00196877019
:1006D00099278093C6018091C60190919501891355
:1006E000E7CF0FC0109270010E94BF0210929501D7
:1006F0001092C601EFE8F1E086E0DF011D928A95D5
:10070000E9F767960FB6F894DEBF0FBECDBFDF9155
:10071000CF9108958F929F92AF92BF92CF92DF9226
:10072000EF92FF920F931F93CF93DF93CDB7DEB776
:100730002A970FB6F894DEBF0FBECDBFFC01008133
:10074000D18083819481892B39F02FEFD21206C09A
:1007500091E00F3F19F403C091E001C090E090FDDB
:100760003FC27F0185E0DE01169601900D928A95C9
:10077000E1F7F70122818E819F81222349F00E94B7
:100780005802182F682F8E819F810E943E0103C05E
:100790000E941501182F812F90E063E070E00E9405
:1007A00053148D0D911DFC01EE0FFF1FEE0FFF1F67
:1007B000E00FF11DEE0FFF1FE356FE4F2591349120
:1007C000F70182818823E1F12115FCE53F07B9F0AB
:1007D0002F3D3C45A9F52A960FB6F894DEBF0FBE13
:1007E000CDBFDF91CF911F910F91FF90EF90DF90E0
:1007F000CF90BF90AF909F908F900C94830E1092EB
:1008000070010E94BF025FEF84E39CE05150804082
:100810009040E1F700C000002A960FB6F894DEBFC2
:100820000FBECDBFDF91CF911F910F91FF90EF9041
:10083000DF90CF90BF90AF909F908F900C94290B3A
:10084000F70110810181882359F0812F902F0E9498
:100850005802D82E682F812F902F0E943E0105C08C
:10086000812F902F0E941501D82E8D2D90E063E0EE
:1008700070E00E945314800F911DFC01EE0FFF1FCA
:10088000EE0FFF1FE10FF11DEE0FFF1FE356FE4FAE
:10089000859194910E94030D082FC82EF7012281A3
:1008A0004581342F32953F70D92ED2945FE0D52206
:1008B0008D2C912CFCE08F16910408F069C1F40195
:1008C000E65CFF4F0C947814892F807F9F70192F5E
:1008D000882311F01295107F2223B9F0112309F417
:1008E00043C180E2800F883010F0C11006C09091A3
:1008F0007001192B1093700105C09091CF01192B35
:100900001093CF010E94E80E2FC1802F0E94A801F2
:10091000112309F43DC1005E1095083010F0C1109C
:1009200006C09091700119231093700105C0909139
:10093000CF0119231093CF010E94E80E29C1592F2E
:10094000507F892F8F70503211F08295807F51E057
:10095000C5120AC0222321F0363008F019C10DC09B
:10096000353008F015C119C0222351F0332329F086
:1009700040FFFAC04F70F70145830E94770108C11C
:10098000332359F0093309F000C1FFEF27EE43E0AC
:10099000F15020404040E1F7F6C00E946C01F8C0E1
:1009A000892F86958695837019F0813059F0F0C0B3
:1009B000222319F0802F937002C080E090E00E9403
:1009C000BE0BECC0222319F0802F937002C080E090
:1009D00090E00E94A80BE2C0892F8370A9F5211135
:1009E000DBC0802F829586958770880F880F202F17
:1009F0002F70082E01C0220F0A94EAF704FF09C0E5
:100A00004FE050E001C0440F8A95EAF7842F8095AB
:100A100001C080E096959695492F4370423069F069
:100A200088F49091D001413019F0822B892302C0C3
:100A3000922B892B0E949B02AFC0822B9091D001F8
:100A40008927F8CF822BF6CF222319F0892F8170C6
:100A500001C08695882309F49FC0802F82958695D2
:100A60008770880F880F202F2F70082E01C0220F4B
:100A70000A94EAF704FF09C04FE050E001C0440FB8
:100A80008A95EAF7842F809501C080E09695969527
:100A9000492F4370423059F078F49091D801413099
:100AA00019F0822B892309C0922B892B06C0822B37
:100AB0009091D801892701C0822B0E948D016CC0C2
:100AC000192F1F70222339F0812F0E949D01802F42
:100AD0000E94770161C00E946C01812F0E949101E8
:100AE0005BC051EF851709F1581720F0E0EF8E1722
:100AF00041F036C0F2EF8F17F9F043EF841719F188
:100B00002FC0222379F0353008F042C0292F2F71F1
:100B100081E090E001C0880F2A95EAF79091D80112
:100B200089271BC03630A0F5F1CF222339F0892F59
:100B30008F710E949D012CC02223C9F3892F8F71D0
:100B40000E94910125C0222339F09F7181E001C0EC
:100B5000880F9A95EAF701C080E00E948D0118C0C5
:100B6000222331F0332319F3802F0E94E00110C0BB
:100B7000332321F3893349F45FEF87EE93E051503B
:100B800080409040E1F700C00000802F0E94A80143
:100B900088EF8D0D843010F40E94D40B85E0F701AE
:100BA000DE01119601900D928A95E1F789819A8173
:100BB0000E94150190E063E070E00E9453142A81C6
:100BC000820F911DFC01EE0FFF1FEE0FFF1F8981A9
:100BD000E80FF11DEE0FFF1FE356FE4F8591949134
:100BE0002A960FB6F894DEBF0FBECDBFDF91CF912E
:100BF0001F910F91FF90EF90DF90CF90BF90AF903B
:100C00009F908F9008952091E4003091E50095E643
:100C10004091EC00842F817040FF23C08091E80058
:100C200080FD1DC080917D01882399F0853099F069
:100C30008091EB0085FD11C04091E4005091E500EA
:100C40002417350729F3915011F09A01E1CF84E080
:100C5000089582E0089583E0089581E0089580E09A
:100C600008954091E80042FFDDCF0895EF92FF9292
:100C70000F931F93CF93DF937C018B010E94030698
:100C8000811119C0E70101151105A1F08091E8005B
:100C900085FD0AC08091E8008E778093E8000E946D
:100CA0000306882381F307C089918093F1000150E6
:100CB0001109E9CF80E0DF91CF911F910F91FF9053
:100CC000EF90089580917F0187FF11C08091E80027
:100CD00082FD05C080917D018111F8CF11C0809106
:100CE000E8008B770BC080917D01882349F08091CB
:100CF000E80080FFF8CF8091E8008E778093E800CD
:100D0000089520918501309186012617370748F014
:100D10006115710539F42091E8002E772093E800E1
:100D200001C0B901FC0120E06115710561F18091FC
:100D30007D018823D9F18530D9F18091E80083FDC8
:100D400039C08091E80082FD2BC08091E80080FFCF
:100D5000EBCF8091F20090E06115710551F0883081
:100D6000910538F421912093F100615071090196A9
:100D7000F3CF21E0089709F020E08091E8008E771A
:100D80008093E800D1CF2111D2CF0AC080917D019C
:100D9000882361F0853061F08091E80083FD0AC00E
:100DA0008091E80082FFF2CF80E0089582E008950C
:100DB00083E0089581E00895089508958091720177
:100DC000089580936D0170936F0160936E0180911F
:100DD0007D01843001F582E08093E9008FEF9091EE
:100DE000E800815095FD06C095ED9A95F1F7000059
:100DF0008111F5CF8091E80085FF0DC040E050E003
:100E000063E070E08DE691E00E9436068091E80094
:100E10008E778093E8000895BC0184E00C94E1068D
:100E2000BC0183E00C94E106CF93DF9321E0209393
:100E3000E9002FEF3091E800215035FD06C035ED77
:100E40003A95F1F700002111F5CF2091E80025FF38
:100E500014C0EC0140E050E068E070E00E9436060B
:100E60008091E8008E778093E80088E0FE01A3E798
:100E7000B1E001900D928A95E1F7DF91CF9108954D
:100E8000982F953068F59093E900981739F0709194
:100E9000EC002091ED005091F00003C0242F762F3C
:100EA00050E021FD02C09F5FECCF3091EB003E7F10
:100EB0003093EB003091ED003D7F3093ED003091A9
:100EC000EB0031603093EB007093EC002093ED0069
:100ED0005093F0002091EE0027FDE5CF80E00895CB
:100EE0008F708093E90081E008951F93CF93DF9383
:100EF000CDB7DEB7AA970FB6F894DEBF0FBECDBF51
:100F0000EFE7F1E087E891E02091F10021938E175F
:100F10009F07D1F780918001833009F45DC030F4E0
:100F2000813071F0823009F499C0B0C08A3009F480
:100F300085C08B3009F468C0893009F0A7C020C093
:100F400080917F01813A09F0A1C08091E800877FFC
:100F50008093E8008091830190918401892B21F492
:100F600068E083E791E003C060E080E090E070E03B
:100F70000E9481068091E8008B778093E80086C00C
:100F800080917F01813209F081C08091830190912D
:100F90008401029708F07AC08091E800877F8093EF
:100FA000E8008091E80082FD05C080917D018111FB
:100FB000F8CF6CC08091F200823031F48091F10062
:100FC000813011F0863021F48091F100809372011C
:100FD0008091E8008B7756C080917F01813A09F0BB
:100FE00055C08091830190918401892B09F04EC0F6
:100FF0008091E800877F8093E8008091E80080FF7F
:10100000FCCF8091000139C080917F018132F1F5E0
:101010008091830190918401892BC1F58091E80032
:10102000877F8093E8000E9462068091810180930F
:101030000001109270010E94BF0228C080917F01C0
:10104000813221F58091E800877F8093E8000E943B
:101050006206809182018093710118C080917F01A6
:10106000813AA1F48091E800877F8093E800809125
:10107000E80080FFFCCF809171018093F1008091A6
:10108000E8008E778093E8000E9462068091E80075
:1010900083FFCAC180917F0190918001492F50E068
:1010A0004A30510508F0C0C1FA01EA5BFF4F0C94C9
:1010B0007814803821F0823809F0B6C108C08091D8
:1010C0007B0190917C01992389F082600FC080910F
:1010D00083018F70853008F0A7C18093E90080916B
:1010E000EB0085FB882780F91092E9009091E800D9
:1010F000977F9093E8008093F1001092F10061C116
:10110000282F2D7F09F090C1882319F0823061F0DB
:101110008BC180918101813009F086C1933009F043
:1011200080E080937C012EC08091810181112AC0D2
:10113000809183018F702FEF280F243008F074C145
:101140008093E9002091EB0020FF1CC0933021F434
:101150008091EB00806214C09091EB0090619093BD
:10116000EB0021E030E0A90102C0440F551F8A9531
:10117000E2F74093EA001092EA008091EB00886069
:101180008093EB001092E9008091E800877F1CC1FA
:1011900081114AC1109181011F778091E30080780D
:1011A000812B8093E3008091E800877F8093E800A3
:1011B0000E9462068091E80080FFFCCF8091E300EE
:1011C00080688093E300111102C082E001C083E0D7
:1011D00080937D0129C18058823008F025C180911B
:1011E0008101909182018C3D53E0950779F583E070
:1011F0008A838AE289834FB7F894DE01139620E050
:101200003EE051E2E32FF0E050935700E49120FFDD
:1012100003C0E295EF703F5FEF708E2F90E0EA30F1
:1012200010F0C79601C0C0968D939D932F5F243117
:1012300049F74FBF8091E800877F8093E8006AE21A
:1012400070E0CE0101960E948106AAC04091830100
:1012500050918401292F332723303105A9F068F4F8
:101260002130310509F4EFC02230310509F0DCC02E
:101270008BE390E0E2E1F1E044C02132310521F15D
:101280002232310571F1D0C0992781309105A1F04A
:1012900058F0029709F0C8C0EFE5F1E0E4918E2F15
:1012A00090E0EFE5F1E02AC0E9E9F1E0E4918E2F6A
:1012B00090E0E9E9F1E022C0E3E8F1E0E4918E2F6B
:1012C00090E0E3E8F1E01AC04115510509F4C0C00F
:1012D0004130510509F0A8C089E090E0EDE3F1E06C
:1012E00010C04115510509F4B8C04130510509F04D
:1012F0009BC082E390E0E0EAF0E003C0009709F4CD
:1013000093C02091E800277F2093E8002091850179
:10131000309186018217930708F49C0140E0211563
:10132000310569F180917D018823D1F18530C1F1CA
:101330008091E80083FD34C08091E80082FD2CC0DC
:101340008091E80080FFEBCF8091F20090E02115C2
:10135000310559F08830910540F444914093F100F3
:101360003196215031090196F2CF41E0089709F0FA
:1013700040E08091E8008E778093E800D0CF411163
:10138000D1CF0AC080917D01882351F0853041F092
:101390008091E80083FD04C08091E80082FFF2CFD5
:1013A0008091E8008B778093E8003EC08038E1F5BB
:1013B0008091E800877F8093E80080917E01809390
:1013C000F1008091E8008E778093E8000E94620629
:1013D0002BC0811129C080918101909182019927B0
:1013E000029714F58091E800877F8093E8001091C0
:1013F000810110937E010E946206111106C0809146
:10140000E30087FD02C081E001C084E080937D019C
:1014100042E061EC81E00E94400742E261EC82E040
:101420000E94400780917D018091E80083FF1AC0EF
:101430008091E800877F8093E8008091EB008062D4
:101440008093EB000FC082E190E0EDE4F1E059CF32
:1014500089E090E0E4E2F1E054CF80E490E0E2ED56
:10146000F0E04FCFAA960FB6F894DEBF0FBECDBF07
:10147000DF91CF911F9108951F920F920FB60F9297
:1014800011242F933F934F935F936F937F938F9389
:101490009F93AF93BF93CF93DF93EF93FF93C0914D
:1014A000E900CF708091EC00D82FD17080FDD0E89A
:1014B0001092E9008091F000877F8093F00078948B
:1014C0000E9475071092E9008091F0008860809377
:1014D000F000CD2BCF70C093E900FF91EF91DF9129
:1014E000CF91BF91AF919F918F917F916F915F91BC
:1014F0004F913F912F910F900FBE0F901F90189515
:101500001F920F920FB60F9211242F933F934F9378
:101510005F936F937F938F939F93AF93BF93EF935B
:10152000FF938091E10082FF09C08091E20082FF79
:1015300005C08091E1008B7F8093E1008091E10004
:1015400080FF17C08091E20080FF13C08091E2000D
:101550008E7F8093E2008091E20080618093E200C0
:101560008091D80080628093D80019BC85E0809378
:101570007D018091E10084FF30C08091E20084FF12
:101580002CC084E089BD86E089BD09B400FEFDCF92
:101590008091D8008F7D8093D8008091E1008F7E6C
:1015A0008093E1008091E2008F7E8093E200809141
:1015B000E20081608093E20080917E01882311F037
:1015C00084E007C08091E30087FD02C081E001C094
:1015D00083E080937D0180917D018091E10083FF14
:1015E00027C08091E20083FF23C08091E100877FC4
:1015F0008093E10082E080937D0110927E018091D2
:10160000E1008E7F8093E1008091E2008E7F8093E5
:10161000E2008091E20080618093E20042E060E0BD
:1016200080E00E9440078091F00088608093F00085
:10163000FF91EF91BF91AF919F918F917F916F91AA
:101640005F914F913F912F910F900FBE0F901F9080
:10165000189581E08093E00080E28093D80010929A
:10166000C9008FE19EE40197F1F700C0000087E018
:1016700090EBDC018093E9019093EA01A093EB01E8
:10168000B093EC019CE088E10FB6F894A8958093A4
:1016900060000FBE90936000FFCF78941F920F926E
:1016A0000FB60F9211248F939F93AF93BF938091A6
:1016B000690190916A01A0916B01B0916C01019652
:1016C000A11DB11D8093690190936A01A0936B01E4
:1016D000B0936C01BF91AF919F918F910F900FBE0E
:1016E0000F901F9018952FB7F894809169019091F1
:1016F0006A01A0916B01B0916C012FBF08951F92F8
:101700000F920FB60F9211248F939F93AF93BF93B5
:1017100080916801811113C08091690190916A01E3
:10172000A0916B01B0916C014196A11DB11D8093F8
:10173000690190936A01A0936B01B0936C01BF9112
:10174000AF919F918F910F900FBE0F901F901895A2
:1017500020916601309167012817390771F0909345
:10176000670180936601E0916401F0916501309713
:1017700021F00084F185E02D099408952091620103
:10178000309163012817390771F0909363018093BA
:101790006201E0916401F0916501309721F00680CB
:1017A000F781E02D09940895E0916401F0916501BD
:1017B000309721F00190F081E02D099480E00895A8
:1017C00080E008959091D90192FF0DC0282F2871D3
:1017D000283019F4877F846006C0282F24712430B4
:1017E00011F48B7F886093FF0DC0282F287128315A
:1017F00019F4877E846106C0282F2471243111F4E6
:101800008B7E88612091DA0120FF0DC0382F38715E
:10181000383019F4877F816006C0382F317131303C
:1018200011F48E7F886021FF0DC0282F2871283188
:1018300019F4877E816106C0282F2171213111F4AE
:101840008E7E886194FD877E0895F894E82FE29556
:10185000EF70F0E031A1282F2F7081E090E001C0FF
:10186000880F2A95EAF7982F9095932391A392A138
:10187000892B82A3789408957F928F929F92AF9242
:10188000BF92CF92DF92EF92FF920F931F93CF936D
:10189000DF9300D01F92CDB7DEB719821A821B8268
:1018A0000EE311E0AE014F5F5F4F7A014A01CC2495
:1018B000C394D12C95E4A92E91E0B92EF801808132
:1018C0008F3F09F440C0F894E82FE295EF70F0E004
:1018D00021A18F70A60102C0440F551F8A95E2F71F
:1018E000CA01922F982B91A392A18095892382A35C
:1018F000789400C0E1E4F1E0712C31E021912F3FB8
:1019000089F0A22FA295AF70B0E090968C9190E0F4
:101910002F7002C0959587952A95E2F780FD02C049
:10192000832F01C080E0782A330FAE16BF0631F74F
:10193000F80180818F3F11F00E94250CF0EAFA95A2
:10194000F1F7F70170820F5F1F4FFFEFEF1AFF0AE9
:1019500041E00134140709F0B1CF43E050E0B40195
:1019600085ED91E00E94921411E0009709F410E0D7
:10197000892B91F089819A81AB818093D5019093D5
:10198000D601A093D70181E08093D3010E94730B0D
:101990009093D2018093D1018091D301882309F1E2
:1019A0002091D1013091D2014FB7F8948091690113
:1019B00090916A01A0916B01B0916C014FBF821BA5
:1019C000930B059770F08091D5018093DB01809196
:1019D000D6018093DC018091D7018093DD011092C4
:1019E000D301812F0F900F900F90DF91CF911F9116
:1019F0000F91FF90EF90DF90CF90BF90AF909F90AE
:101A00008F907F900895CF93DF938238910569F18D
:101A1000B0F48133910509F46FC048F4893291051F
:101A200009F465C08A32910509F46BC08AC0853318
:101A3000910509F457C089339105B9F082C0833EFE
:101A4000910571F138F4803E9105B1F0823E910527
:101A500011F177C0863E9105B9F1873E9105C9F134
:101A6000843E910509F06DC024C02091D90120FD6C
:101A700053C021FD51C065C08091D90180FD46C091
:101A80008091DA0180FF48C08091D90184FD36C180
:101A900083EE90E035C18091D90182FF3AC0F4CF46
:101AA0008091D90182FD35C08091DA0180FD34C07A
:101AB000EBCF8091DA0181FF35C08091D90184FD9F
:101AC0001DC187EE90E01CC18091D90183FF27C022
:101AD000F4CF8091D90183FD22C08091DA0181FD8C
:101AE00021C0EBCF8091D90185FD1FC021C080911D
:101AF000D90185FD1DC019C08091D90186FD1BC08B
:101B00001DC08091D90186FD19C015C089E390E000
:101B1000F7C082EE90E0F4C080EE90E0F1C086EE77
:101B200090E0EEC084EE90E0EBC089E290E0E8C087
:101B300085E390E0E5C08AE290E0E2C081E390E0D6
:101B4000DFC0811531E5930708F064C0811520E5F9
:101B5000920700F19C0174E0369527957A95E1F79C
:101B60002370982F937041E050E002C0440F551F3E
:101B70009A95E2F75C68522B282F2F7026952695B0
:101B800030E0C901E5E0880F991FEA95E1F7842B61
:101B9000952BB6C08F3B910520F5883A910558F0FA
:101BA000885AE82FF0E0EE0FFF1FE05FFE4F8081C4
:101BB00091819464A5C0853A910548F0855AE82F33
:101BC000F0E0E35FFE4F808190E0906499C0843044
:101BD000910508F095C0019709F090C081E090E070
:101BE0008FC0811530E2930768F4811521E09207D8
:101BF00008F086C09C01205E31092830310508F0CC
:101C00007DC07EC0811530E4930708F477C09F70D3
:101C1000906A76C0811524E59207E8F5811533E5D1
:101C20009307C0F0AC014370552721E030E002C0BB
:101C3000220F331F4A95E2F7982F96959695892F94
:101C400090E045E0880F991F4A95E1F7822B932B8E
:101C50009A6856C0811522E5920728F4982F8827A4
:101C6000816F906A4DC0AC014370552721E030E090
:101C700002C0220F331F4A95E2F7982F969596954A
:101C8000892F90E055E0880F991F5A95E1F7822B34
:101C9000932B9C6835C0EC0181153AE59307F8F465
:101CA000C11589E5D80790F08C2F8F700E94E20B48
:101CB00094E0D695C7959A95E1F7CF70D0E0DC2FE8
:101CC000CC27D0699E01282BC9011AC0C11528E56F
:101CD000D207A0F09C2F8827806F906A11C0905681
:101CE0008115904258F48D2F8F710E94E20B282F9E
:101CF0002F71CE0199279062922B02C080E090E074
:101D0000DF91CF91089569EE7EEF80E090E00E9430
:101D10003D1460E082E090E00E941F1460E083E0E8
:101D200090E00E941F141092D00160E084E090E0E7
:101D30000E941F1460E082E290E00E941F1460E0A5
:101D400085E090E00E941F1460E086E090E00E9431
:101D50001F146FEF87E090E00E941F1440E050E0F6
:101D6000BA0188E090E00E94311460E08DE090E0DC
:101D70000E941F1440E050E0BA0188E190E00E9408
:101D8000311460E087E190E00E941F1440E050E0D1
:101D9000BA018CE190E00E94311460E070E080E2D2
:101DA00090E00E943D1440E050E0BA0188E190E0EC
:101DB0000E94311440E050E0BA018FE090E00E94B0
:101DC000311440E050E0BA0183E190E00C9431140A
:101DD000909170018091CF01892B8093870148E019
:101DE00050E067EC71E087E891E00E949214892B43
:101DF000A9F088E0E7E8F1E0A7ECB1E001900D92EE
:101E00008A95E1F7E0916401F0916501309731F036
:101E10000280F381E02D87E891E009940895809194
:101E2000C60190919501891719F08F5F8770FBCFDC
:101E300008951F93CF93DF938091940182958F70C3
:101E400009F05CC080919101882309F457C020916A
:101E5000C60110919501C0918F01D0919001A09180
:101E60009201B091930181E0CF3F09F080E0482FCB
:101E7000211709F443C0109721F0DF3F21F080E0E3
:101E800003C081E001C0842F30E080FD33C0C90170
:101E900066E070E00E945314FC01EA56FE4F818117
:101EA0008D1328C080818C1325C08281811122C0AE
:101EB000838194818A1B9B0B883C9105D8F4809187
:101EC00094018F70806180939401C90166E070E095
:101ED0000E945314FC01E556FE4F90819F70906163
:101EE00090838FE891E00E948A03DF91CF911F9148
:101EF0000C940F0F2F5F3F4F2770BACFDF91CF9118
:101F00001F910895CF93DF93EC010E94580290E057
:101F100063E070E00E9453148D0F911DFC01EE0FE1
:101F2000FF1FEE0FFF1FEC0FF11DEE0FFF1FE3561B
:101F3000FE4F859194910E94030DDF91CF910895FA
:101F40009F92AF92BF92CF92DF92EF92FF920F9348
:101F50001F93CF93DF93CDB7DEB761970FB6F89499
:101F6000DEBF0FBECDBF8C0185E0F801DE011D96FE
:101F700001900D928A95E1F7D8011296EC9090911C
:101F80008F01509190012091920130919301211580
:101F9000310531F05F3F31F481E09F3F19F403C018
:101FA00081E001C080E0B82FB1709B2E80FD27C179
:101FB000D801EC9111964C9111971396CD90DC902D
:101FC00014978FE8A82E81E0B82EF0909101B60109
:101FD000621B730BFF2009F4CCC080919401683C14
:101FE000710508F096C0282F207F09F055C05413C2
:101FF00012C09E1310C0FE2CE1100DC08F708061C6
:1020000080939401C5010E948A0380919401D801B4
:1020100015968C9331C1CD2831F04F3F31F481E0DA
:10202000EF3F19F403C081E001C080E080FD03C0F0
:1020300081E08E2502C080E090E0B82FB170FB2EC9
:1020400080FF20C02091C601F09195012F1709F45F
:10205000F1C030E0C90166E070E00E945314DC0179
:10206000AA56BE4F11968C911197481307C08C91B8
:102070008E1304C012968C91E81204C02F5F3F4F5C
:102080002770E4CFFE2CEE2009F4F6C08091940175
:1020900081608093940149C0541306C09E1304C00C
:1020A000E11002C0D80189C0C8010E949F028823A4
:1020B00051F1EE2041F120919401822F82958F7091
:1020C00090E0029774F080918F0190919001988731
:1020D0008F831986DB86CA862C87CE0107960E94DD
:1020E0008A0386E0F801AFE8B1E001900D928A958D
:1020F000E1F70E94190F0AC05417C9F0C8010E94E5
:102100009F0281111FC0C8010E948A03FF24F3941B
:10211000B3C0282F207F81F78FE891E00E948A03C7
:1021200086E0F50111928A95E9F7F12CA5C09E137E
:10213000E5CFE110E3CFD80115968C93C8010E943A
:102140008A0357C0EE20F9F220919401822F8295E4
:102150008F7090E002972CF280918F019091900106
:102160009A8389831B82DD82CC822E83CE010196E5
:10217000B6CF683C7105E8F5FE2CEE2021F2541331
:102180002AC09E1328C02091940120FD1BC0822FDD
:1021900082958F70482F50E04115510599F0D80174
:1021A00015962C9315974F30510549F08F5F982F56
:1021B0009295907F822F8F70892B15968C93C801F2
:1021C0000E948A0386E0F801AFE8B1E001900D9229
:1021D0008A95E1F751C0C8010E949F02811181CF09
:1021E00080919401816080939401C8010E948A03C8
:1021F00043C086E0F50111928A95E9F73DC0EE20D3
:1022000009F481CFC8010E949F02F82E882309F4A7
:102210007ACF86E0F801AFE8B1E001900D928A959F
:10222000E1F780918F01909190010E94820F0E94AE
:10223000190F22C0ED874E878D859E850E94820FE3
:10224000292F22952F70223028F49F7039F08111A8
:1022500005C00BC0243028F49F7049F4805E88309C
:1022600020F0C8010E948A039F2CF92C05C0F801B8
:102270009581907F99F7F9CF8F2D61960FB6F894DD
:10228000DEBF0FBECDBFDF91CF911F910F91FF90A9
:10229000EF90DF90CF90BF90AF909F900895CF9335
:1022A000DF93CDB7DEB72A970FB6F894DEBF0FBE27
:1022B000CDBF84B7877F84BF0FB6F894A89580916F
:1022C0006000886180936000109260000FBE90E013
:1022D00080E80FB6F89480936100909361000FBE80
:1022E00080EE9BE090935B0180935A011092E20094
:1022F0001092E1008091E00081608093E000809185
:10230000D8008F778093D80019BC809163008160DA
:10231000809363001092D401809163008E7F80933C
:10232000630081E08093D4011092E2001092E100FA
:102330008091D8008F778093D8008091D8008068F2
:102340008093D8008091D8008F7D8093D80084E05E
:1023500089BD86E089BD09B400FEFDCF10927D01E4
:1023600010927E0110927C0110927B0142E060E0AD
:1023700080E00E9440078091E1008E7F8093E10021
:102380008091E20081608093E2008091E2008860A9
:102390008093E2008091E0008E7F8093E000809146
:1023A000E20084608093E200789480917D0188232C
:1023B000A1F01091E9001F709091EC00892F8170BD
:1023C00090FD80E8182B1092E9008091E80083FDD1
:1023D0000E9475071F701093E90082E084BD93E0AE
:1023E00095BD9AEF97BD80936E0080E30E94250C07
:1023F00081E30E94250C82E30E94250C01E411E098
:1024000065E4E62E61E0F62ED8018D918D018F3FB7
:1024100011F00E94250CE016F106B1F783E0EBED18
:10242000F1E0DF01E82E1D92EA94E9F7E5EDF1E035
:10243000DF011D928A95E9F780E090E00E9419146F
:10244000893E9E4F11F00E94830E82E090E00E9430
:1024500011148093DE0184E090E00E941114182F83
:1024600082E290E00E941114212F30E0382B30934B
:10247000DA012093D9010E943C0CEFE3FCE931978B
:10248000F1F700C000000E943C0C8091DD0180FF4C
:1024900008C06FEF7FEF80E090E00E943D140E9443
:1024A000290B83E090E00E9411140E949B0269E5D1
:1024B00071E025E531E0A7E5B1E041E050E06A17C1
:1024C0007B0769F18D91E82FE295EF70F0E011A1A3
:1024D0008F707A0102C0EE0CFF1C8A95E2F7C701EB
:1024E0009E2D9095912391A392A1892B82A3F9010E
:1024F00081919F01E82FE295EF70F0E011A18F70BC
:102500007A0102C0EE0CFF1C8A95E2F7C7019E2DEE
:102510009095912391A392A1892B82A3D0CF8FE88C
:1025200091E00197F1F700C0000089B181704999ED
:1025300002C090E001C092E0892B8093E60189B14E
:1025400082FB882780F94B9902C090E001C092E09D
:10255000892B8093E70181E091E09093650180935E
:10256000640154E0452E512C80917D01853009F0A5
:1025700049C016E080917D01853009F03DC0809111
:102580007D01843021F110926801A8E1B0E0E0E41F
:102590000FB6F894A895A09360000FBEE09360007A
:1025A00083B7817F846083BF83B7816083BF789462
:1025B000889583B78E7F83BF0FB6F894A8958091D6
:1025C0006000886180936000109260000FBE80916F
:1025D0007C01882309F4CECF0E943C0C8091DB0162
:1025E000811105C18091DC01811101C18091DD0162
:1025F000882309F4BFCFFBC0109270010E94BF0274
:102600000E94D40B0E943C0C882359F08FB7F89499
:102610004091690150916A0160916B0170916C0168
:102620008FBFABEDB1E0EFEDF1E000E010E0302F57
:102630002D919191922721F180E0FF24F3944F2D69
:102640004923D1F089833A832F2181E009F480E086
:102650008B830E94730B8160782F9D838C834981CB
:102660005A816B818D810E94DF02F801E152FE4F99
:102670008081F826F08219C08F5FFF0C8430F9F654
:102680000F5F1F4F0330110591F68FEF8E838F83FD
:1026900018860E94730B8160782F9A8789874E81F4
:1026A0005F8168858A850E94DF0296EEA92E91E0FF
:1026B000B92E24EEE22E21E0F22E02EE11E035E5F5
:1026C000C32E31E0D32E47E5642E41E0742E450140
:1026D000212C312CD4018D914D01E82FEE0FEE0FFE
:1026E000D3012D913D01A22FA295AF70B0E090963D
:1026F0008C9190E02F7002C0959587952A95E2F70E
:102700009C0121703327D6018D916D01A82FA295D0
:10271000AF70B0E090964C9150E08F7002C055952C
:1027200047958A95E2F7CA018170992740FF02C058
:1027300082E090E0822B932B8E2BF50181935F0139
:102740008F70E82FF0E0EB5BFE4F9081D7018C910A
:10275000890F8C9384307CF0F80180818F5F8083B7
:1027600060E070E0311002C08EE401C08AEA0E948D
:10277000C80221E001C020E0D7018C918D3F74F4A4
:10278000F80180818150808360E070E0311002C0E8
:102790008BE401C089EA0E94C80221E0D7018C9134
:1027A000082E000C990BB2010E946414F70181936A
:1027B0007F01222A33940F5F1F4FF2E03F128ACF2E
:1027C000222059F08FB7F8944091690150916A0125
:1027D00060916B0170916C018FBF0E94D40B90913E
:1027E000E801891709F4C0CE8093E801BDCE84E0EA
:1027F000E82EE9BC19BD09B400FEFDCF8091D800D8
:102800008F7D8093D8008091E00082608093E0000B
:102810008091E00081FDFCCF109270010E94BF0208
:10282000A9CEF999FECF92BD81BDF89A992780B5BE
:102830000895A8E1B0E042E050E00C944514262F42
:10284000F999FECF92BD81BDF89A019700B40216A6
:1028500039F01FBA20BD0FB6F894FA9AF99A0FBE54
:1028600008950396272F0E9420140E941F14252FDD
:102870000E942014242F0C9420140196272F0E94CC
:1028800020140C941F14DC01CB01FC01F999FECF3C
:1028900006C0F2BDE1BDF89A319600B40D924150E8
:1028A0005040B8F708950024552704C0080E591F5A
:1028B000880F991F009729F076956795B8F37105F1
:1028C000B9F7802D952F089597FB072E16F40094E5
:1028D00007D077FD09D00E947E1407FC05D03EF496
:1028E000909581959F4F0895709561957F4F0895BC
:1028F000EE0FFF1F0590F491E02D0994AA1BBB1B5E
:1029000051E107C0AA1FBB1FA617B70710F0A61BEF
:10291000B70B881F991F5A95A9F780959095BC0110
:10292000CD010895FB01DC0104C08D910190801957
:1029300021F441505040C8F7881B990B0895F89432
:02294000FFCFC7
:1029420001DE061407DD0610070C07DC0681828310
:10295200E200E900EA00B500B600B700CD0083014D
:10296200CC008A0192019401210223022402250251
:10297200260227022A02B300B4006F007000303131
:10298200323334353600FF0100010000FFFF000042
:0A299200010001FF009193909200F4
:00000001FF
